:0B213C00011F08C107011DFF011EFF6D
:04002E0043B1402278
:0400460053B1BF22D1
:04004E0063B1402238
:0100320022AB
:01004A002293
:01005200228B
:0113FF0022CB
:012333002287
:10199D00EF5407FE7401A806088002C333D8FCFE7D
:1019AD00EF131313541FFFED601EEF14600E146040
:1019BD000F14601024037031EE428022EE4290220B
:1019CD00EE42A022EE42B022EF14600F146011140B
:1019DD00601324037013EEF4528022EEF452902221
:0919ED00EEF452A022EEF452B017
:0119F60022CE
:101CDF00EF54F824F8601024F8601024F8601024F2
:101CEF0018700EAE80800AAE908006AEA08002AE55
:101CFF00B0EF5407FF7401A807088002C333D8FC64
:0B1D0F005206EE60047F0180027F009E
:011D1A0022A6
:10000E00E5801202F3900001E590120305900002C4
:0D001E00E5A0120305900003E5B002030504
:101F64001202AD902869F0F5809000011202C6902B
:101F7400286AF0F5909000021202C690286BF0F5E2
:0E1F8400A09000031202C690286CF0F5B02267
:10203B0090286874FFF0902867F0902866F090283D
:10204B0065F090286CF090286BF090286AF090283F
:03205B0069F02207
:10178B00E4F5B2F5B3F5B4F5B5902865E0FF9080BC
:10179B0000F0902866E0FE908001F0902867E0FD55
:1017AB00908002F0902868E0FC908003F08FB28E5E
:1017BB00B38DB48CB5902869E0F580A3E0F590A3C8
:1017CB00E0F5A0A3E0F5B0902865E0F4908004F07C
:1017DB00902866E0F4908005F0902867E0F4908004
:1017EB0006F0902868E0F4908007F075B1BF75B6ED
:0217FB00442286
:102289008F628D6330060302104EAD63AF62121088
:022299006D22B4
:012334002286
:012335002285
:0D00360090286D74FFF0A3F0A3F0A3F0225A
:1017FD00E4F5B2F5B3F5B4F5B590286DE0FF908042
:10180D0000F090286EE0FE908001F090286FE0FDD2
:10181D00908002F0902870E0FC908003F08FB28EE3
:10182D00B38DB48CB5902871E0F580A3E0F590A34D
:10183D00E0F5A0A3E0F5B090286DE0F4908004F001
:10184D0090286EE0F4908005F090286FE0F4908081
:0C185D0006F0902870E0F4908007F02264
:10127400A980AD90E51D69F522E51E6DF5231200E8
:101284002EE5225523F524E4FCECC3951F4003020C
:10129400134A7401A804088002C333D8FCFFE52272
:1012A40060365F6033E95F6006ED5F60068016EDCF
:1012B4005F6012EC25E02475F582E43428F583E4BC
:1012C40075F0018010EC25E02475F582E43428F5EE
:1012D4008374FFF5F012037CE52360365F6033ED21
:1012E4005F6006E95F60068016E95F6012EC25E046
:1012F4002475F582E43428F58374FFF5F08010EC4E
:1013040025E02475F582E43428F583E475F00112B0
:10131400037CE524602C74017E00A804088005C3C6
:1013240033CE33CED8F9FFEF552460047F01800219
:101334007F00EF600D74002CF582E43428F583E01F
:0D13440004F00C02128D891D8D1E02004662
:0D22ED0030070912002E1212741200462252
:1006FD00D204120E5A500302095790E6B9E024EEC7
:10070D0070030208912470700302095014700302E3
:10071D00095024C2600302095590E6B8E020E703B2
:03072D000207FFC1
:10073000E4F529F52AE52A25E02475F582E4342834
:10074000F583A3E0FFAE29052974402EF582E43439
:10075000E7F583EFF0E52A25E02475F582E43428F7
:10076000F583E0FFAE29052974402EF582E434E7D5
:10077000F583EFF07400252AF582E43428F583E050
:10078000FFAE29052974402EF582E434E7F583EFA6
:10079000F074017E00A82A088005C333CE33CED87A
:1007A000F9FF90E6BAE0FDEF5D60047D0180027D17
:1007B00000ED600D7400252AF582E43428F583E409
:1007C000F090E6BCE0FDEF5D60047F0180027F00F9
:1007D000EF6011E52A25E02475F582E43428F583DD
:1007E000E4F0A3F0052AE52A64086003020735E473
:0C07F00090E68AF090E6BEE090E68BF008
:0307FC0002095798
:1007FF0090E6BBE0B4010FA3E0D394085008E09457
:10080F00004003E0F51F90E6BBE0B4021890E6BD90
:10081F00E0FE90E6BCE07C002400FDEC3EFCE41220
:10082F0001F3121F0490E6BBE0700B90E6BAE024D0
:10083F00FF920702095790E6BBE064AC6003020920
:10084F005790E6BAE064CE600302095790E600E0E5
:10085F00F52990E6BCE024E8600D24E86013242419
:10086F0070175329E78012E52954E74408F52980CA
:0F087F0008E52954E74410F52990E600E529F033
:10088E00020957E490E68AF090E6BEE090E68BF01F
:10089E0090E6A0E020E1F9E4F5B2F5B3F5B4F5B5D4
:1008AE0090E744E0902865F0908000F090E745E0F6
:1008BE00902866F0908001F090E746E0902867F06F
:1008CE00908002F090E747E0902868F0908003F067
:1008DE0090E744E0F5B2A3E0F5B3A3E0F5B4A3E0EE
:1008EE00F5B590E740E0902869F0F58090E741E09B
:1008FE0090286AF0F59090E742E090286BF0F5A012
:10090E0090E743E090286CF0F5B090E744E0F49067
:10091E008004F090E745E0F4908005F090E746E023
:10092E00F4908006F090E747E0F4908007F090E6B0
:10093E00BAE025E025E05404FFE5B154FB4FF5B1D4
:0B094E008007120B7E8002D322C32220
:100F7E00120100020000004005160480010001026B
:100F8E0000010A06000200000040010009022000D4
:100F9E00010100A0FA0904000002FF00000007058D
:100FAE00020200020007058602000200090220006C
:100FBE00010100A0FA0904000002FF00000007056D
:100FCE0001024000000705810240000014030000EA
:100FDE000000000000000000000000000000000003
:100FEE002603410043004300450053002000490002
:100FFE002F004F002000500072006F00640075003B
:10100E0063007400730018035500530042002D0056
:10101E00440049004F002D0033003200490000000B
:10102E0080818283848586879091929394959697FA
:10103E00A0A1A2A3A4A5A6A7B0B1B2B3B4B5B6B7EA
:10104E00C0D0C0E0EF90102E93901065F0ED901090
:10105E002E93901067F0A2009200D0E0D0D022C064
:10106E00D0C0E0EF90102E93901084F0ED90102EE3
:0F107E0093901087F0A200B39200D0E0D0D02260
:1021E4005641707220323520323031364031303A27
:0B21F40032313A3036000000000000DD
:10214700025621FB024000000148010144010142FF
:012157000186
:1021FF0090280BE0FF700690280AE0600890280AEC
:09220F00E0FD02217512232622D4
:102081007E007F6D7D007B017A2879081203C6905E
:1020910028087409F0E4A3F012203B12178B0220E8
:0120A100C27C
:102159007D02121AF2902808E0B40904A3E0600392
:0C2169000220817D6D121AF212178B22E9
:1020C2009028087409F0E4A3F07A287B087D6D7FDC
:0F20D200017E1F121E377D6D7F007E1F022323AC
:101869001221FF90E6BEE0F531753302E53160578C
:10187900C3944050058531328003753240E490E6C7
:101889008AF090E68BE532F090E6A0E020E1F9E4F9
:10189900F530E530C39532502574402530F582E4A2
:1018A90034E7F583E0FFAE330533EE7C007B01249A
:1018B90008F9EC3428FAEF1202F3053080D4C3E5B5
:0A18C900319532F53180A50221FFB0
:1013510090E6B8E030E745E4F531F530E530C39487
:101361000850247E007B0174652530F9EE3428FA9B
:101371001202ADFF74402531F582E434E7F583EFC5
:10138100F00530053180D5E490E68AF090E6BEE0C4
:1013910090E68BF090E6A0E04480F02290E6BEE07B
:1013A10090E68BF090E6A0E020E1F990E6BEE064E3
:1013B100086003C20422E4F530F531E530C3940836
:1013C100502474402531F582E434E7F583E0FFE5EC
:1013D100307C007B012465F9EC3428FAEF1202F32A
:1013E1000530053180D590E6BAE0B4CE08A3E0B46B
:0513F100AC031220C254
:0113F60022D4
:0F22CF00D3E5599546E558954540031222DE2286
:012336002284
:10205E0090280DE0FE90280CE07C002400F546EC64
:10206E003EF54545467007C28CC2A9C20522D28CE8
:03207E00D2A922C2
:012337002283
:101C1F0090E6BEE090E68BF090E6A0E020E1F9E4DC
:101C2F00FF74422FF582E434E7F583E0FEEF7C008A
:101C3F007B01246DF9EC3428FAEE1202F30FBF0882
:101C4F00E090E740E090280CF090E741E090280DFD
:041C5F00F002205E11
:0F22DE001217FDE4F54BF54CF558F559D20522D2
:10210000C205E4F54BF54CF558F559C28CC2A953FC
:0E2110008EF75389F143890112233702205EB6
:101D1B00E54145406019E54115417002154014C37A
:101D2B0094FFE54064809480501C1200468017306D
:101D3B0004147540057541FF12002EC204E4F54BE7
:0B1D4B00F54CF558F559300502D204A4
:011D5600226A
:100D1F0090E6B8E020E703020DD4E4F53190280CFB
:100D2F00E0FFAE31053174402EF582E434E7F583F0
:100D3F00EFF090280DE0FFAE31053174402EF582B3
:100D4F00E434E7F583EFF0E4F530E530C394085071
:100D5F00247E007B01746D2530F9EE3428FA1202DF
:100D6F00ADFF74402531F582E434E7F583EFF005EC
:100D7F0030053180D5AE31053174402EF582E43423
:100D8F00E7F583E559F0E558FFAE31053174402E94
:100D9F00F582E434E7F583EFF0A205E433FFAE31DB
:100DAF00053174402EF582E434E7F583EFF0C20588
:100DBF00E490E68AF090E6BEE090E68BF090E6A035
:100DCF00E04480F02290E6BEE090E68BF090E6A043
:100DDF00E020E1F9C20590E6BEE0640A6003C204B8
:100DEF0022E4F531AF31053174402FF582E434E759
:100DFF00F583E090280CF0AF31053174402FF58268
:100E0F00E434E7F583E090280DF0E4F530E530C3E6
:100E1F009408502474402531F582E434E7F583E0DB
:100E2F00FFE5307C007B01246DF9EC3428FAEF12DA
:100E3F0002F30530053180D512205E90E6BAE0B49A
:0A0E4F00CE08A3E0B4AC031220C2E9
:010E59002276
:0423170075480122E2
:1018D3001221FF90E6BEE0F531E4F533E5316057C0
:1018E300C3944050058531328003753240E490E65D
:1018F3008AF090E68BE532F090E6A0E020E1F9E48F
:10190300F530E530C39532502574402530F582E437
:1019130034E7F583E0FFAE330533EE7C007B01242F
:1019230023F9EC3428FAEF1202F3053080D4C3E52F
:07193300319532F53180A56A
:01193A00228A
:101A4E001548E548704B902823E0F548122334E4FE
:101A5E00F55F902864E0FFE55FC39F5031E55F2599
:101A6E00E02424F582E43428F583E0F560E55F2573
:101A7E00E02425F582E43428F583E0F561547FFDFA
:101A8E00E561339206AF60122289055F80C412238E
:011A9E003512
:011A9F002224
:1020A20090E6BEE090E68BF090E6A0E020E1F990A9
:1020B200E740E090280EF090E741E090280FF022F0
:101700001544E544600302178A90280EE0F5447BF7
:10171000017A2879B712000EE4FFFE74B72EF58225
:10172000E43428F583E0FD74852EF582E43428F551
:1017300083E06DF97D01E4FCECC394085046E95D5B
:10174000602974892FF582E43428F583E014F0745D
:10175000892FF582E43428F583E0702074852EF516
:1017600082E43428F583E06DF0800090280FE0FBE0
:1017700074892FF582E43428F583EBF00CED25E035
:0A178000FD0F80B40EEE64047091BA
:01178A00223C
:1022180090E6BEE090E68BF090E6A0E020E1F99031
:08222800E740E0902810F022CD
:101F9200E4FF74A92FF582E43428F583E4F074B3E6
:101FA2002FF582E43428F58374FFF074AF2FF582A5
:0B1FB200E43428F583E4F00FBF04D7EF
:011FBD002201
:10193B001542E542705B902810E0F5427B017A2856
:10194B0079A912000EE4FF74B32FF582E43428F565
:10195B0083C083C082E0FE74A92FF582E43428F59E
:10196B0083E0FDEE5DD082D083F074AF2FF582E47F
:10197B003428F583C083C082E0FE74A92FF582E47E
:10198B003428F583E0FDEE4DD082D083F00FBF04F9
:01199B00B695
:01199C002228
:04231B0075470122DF
:101555001547E547603DE4F564902822E0FFE56422
:10156500C39F507C744E2564F8E6602316E6701F11
:10157500E56425E02412F582E43428F583E0FE5481
:101585007FFFEE30E7047D0080027D0112199D0585
:101595006480C6902811E0F547E4F564902822E0C0
:1015A500FFE564C39F5039E56425E02413F582E423
:1015B5003428F583E0FF744E2564F8A607E5642515
:1015C500E02412F582E43428F583E0FE547FFFEE33
:1015D50030E7047D0180027D0012199D056480BC01
:0115E50022E3
:101EA00090E6BEE090E68BF090E6A0E020E1F9E459
:101EB000FF74402FF582E434E7F583E0FEEF7C0009
:101EC0007B012411F9EC3428FAEE1202F30FBF1251
:011ED000E031
:011ED10022EE
:0414B8008E308F31B2
:1014BC00E4F532E53164024530700C90E741F0E51B
:1014CC0031153170021530E53164014530701690DC
:1014DC00E740746DF090E6BEE090E68BF0E53115D8
:1014EC003170021530E5314530605D90E6A0E020AA
:1014FC00E1F9C3E5319440E53094005004AD3180FE
:10150C00027D40E4FFEFC39D5025AE320532EE75EF
:10151C0083007B012408F9E5833428FA1202ADFE1E
:10152C0074402FF582E434E7F583EEF00F80D6E4B7
:10153C0090E68AF090E68BEDF0FFC3E5319FF53134
:08154C00E5309400F530809DAC
:011554002274
:1003F20090E6B8E030E76390E6BFE0FE90E6BEE04C
:10040200FDEDFF4E7002804D90E6BDE0FD90E6BC32
:10041200E04D70030214B890E6BDE060030206FCF2
:1004220090E6BCE01460030206FC7533FF753421CC
:100432007535E475360075371E7B017AE77941120E
:100442001AA07B017AE77940122274EF0490E74008
:10045200F090E6BEE090E68BF02290E6BFE0FF90DF
:10046200E6BEE04F707790E6BDE0704D90E6BCE0EE
:1004720024EF6023249F603024FD603324F3603432
:100482002472703590E6BAE064CE702DA3E064ACBD
:1004920070271220C2802290E6BAE0B4CE1BA3E0FD
:1004A200B4AC161220818011E4902822F0800A75E3
:1004B20047018005E4902864F090E6BDE064806026
:1004C200030206FC90E6BCE0640160030206FC90B5
:1004D200E6BAE090280AF090E6BB02058F90E6BFEC
:1004E200E060030206FC90E6BDE0FE90E6BCE07C24
:1004F200002400FFEC3E60030206FCEF1203A0059D
:100502003520053521053522053523056A2F059746
:100512004105A55105B35305D36105E16306017198
:10052200060F73062F74068481068F8306AC84003F
:100532000006FC90E6BEE0B46B0312186990E6BCBC
:10054200E030E00312178B90E6BCE020E1030206E4
:10055200FC90E6BAE064CE60030206FCA3E064AC61
:1005620060030206FC0220C290E6BEE06402600361
:100572000206FCE090E68BF090E6A0E020E1F912A2
:1005820021FF90E740E090280AF090E741E09028B0
:100592000BF00221FF90E6BEE0640A60030206FC53
:1005A200021C1F90E6BEE0640260030206FC022009
:1005B200A290E6BEE0640160030206FCE090E68BD6
:1005C200F090E6A0E020E1F990E740E090280EF0FC
:1005D2002290E6BEE0640160030206FC022218904B
:1005E200E6BEE0640160030206FCE090E68BF09058
:1005F200E6A0E020E1F990E740E0902810F0229098
:10060200E6BEE0641260030206FC021EA090E6BE93
:10061200E0640160030206FCE090E68BF090E6A045
:10062200E020E1F990E740E0902811F02290E6BE48
:10063200E0640260030206FC902822E0C3940840B2
:10064200030206FC90E6BEE090E68BF090E6A0E0A6
:1006520020E1F990E740E0FF902822E0FE25E02427
:1006620010F582E43428F583EFF090E741E0FFEEE5
:1006720025E02411F582E43428F583EFF090282256
:10068200807590E6BEE0644270700218D390E6BEB8
:10069200E064017065E090E68BF090E6A0E020E176
:1006A200F990E740E0902823F02290E6BEE0640251
:1006B2007048902864E0C39420503F90E6BEE090DA
:1006C200E68BF090E6A0E020E1F990E740E0FF90B1
:1006D2002864E0FE25E02422F582E43428F583EF45
:1006E200F090E741E0FFEE25E02423F582E4342890
:0A06F200F583EFF0902864E004F0B7
:0106FC0022DB
:1021C90090E6047480F00000007402F000000074CE
:0B21D90006F0000000E4F0000000220F
:012338002282
:101C6300E4F5297AE779407F40AB077D087FF87E6A
:101C73001D121AFAE4F52974402529F582E434E7A4
:101C8300F583E0FDE52975F002A424DCF9740F3532
:0E1C9300F08982F583EDF00529E529B408D922
:011CA1002220
:101D570090E678E05410FFC4540F4450F54913E45B
:101D670033F54D438E2012003212230F121C6312DB
:101D7700004AD200122159122100122317121F9272
:0C1D870012231B1221FF12004602005222
:10211E001213FF121D1B1222CFE5B190E68020E7AD
:0E212E0006E04408F08004E054F7F00223338A
:0619F7008B5A8A5B895C3B
:1019FD00E4F55D1222748F5EE55E25E02402901001
:101A0D0014F0E4F55DAF5EEF3395E0FEC3E55D9F49
:101A1D00EE6480F87480985027AB5AAA5BA95C8558
:101A2D005D827583001202C6FDE55D75F002A4248A
:101A3D0016F9741035F08982F583EDF0055D80C5DA
:011A4D002276
:061B8E008E3E8F3FAC0506
:101B9400E4FDE54D6012E53EFF7E000DEE2557F5B0
:101BA40082E43556F583EFF0AE050DE5572EF58248
:101BB400E43556F583E53FF0AF050DE5572FF58283
:101BC400E43556F583ECF0AB57AA56AF491221AD74
:051BD400AF49021E01F3
:03232300021B8E0C
:0A1E37008E388F398D3A8A3B8B3CC0
:101E4100E4F53DE53DC3953A50200539E539AE3815
:101E51007002053814FFE53C253DF582E4353BF57C
:0A1E610083E0FD122323053D80D924
:011E6B002254
:081AF2007A287B087F017E1FAA
:0A1AFA008E388F398D3A8A3B8B3C01
:101B0400E4FDF53DE54D6012E538FF7E000DEE2560
:101B140057F582E43556F583EFF0AE050DE5572E03
:101B2400F582E43556F583E539F0AB57AA56AF494B
:0E1B34001221ADAB3CAA3BAD3AAF4902219164
:100B7E0090E6BAE0753000F531A3E0FEEE4230901B
:100B8E00E6BEE0753200F533A3E0FEEE423290E6AB
:100B9E00B8E064C06003020C8BE53345327003028B
:100BAE000D1E90E6A0E020E1F9C3E5339440E53256
:100BBE0094005008853234853335800675340075BF
:100BCE00354090E6B9E064A3705890E6BCE0B401FD
:100BDE001BA3E0701790E6BBE030E71090E740747F
:100BEE0003F0A37401F0A37403F0806CE4F536F502
:100BFE0037C3E5379535E5369534505CE531253705
:100C0E00F582E5303536F583E0FF74402537F58201
:100C1E0074E73536F583EFF00537E53770D30536D3
:100C2E0080CFE4F536F537C3E5379535E53695349F
:100C3E00501974402537F58274E73536F58374CD37
:100C4E00F00537E53770E0053680DCAD357AE77BA9
:100C5E0040AF31AE30121AFAE490E68AF090E68B8D
:100C6E00E535F02531F531E5343530F530C3E53372
:100C7E009535F533E5329534F532020BA790E6B88B
:100C8E00E064406003020D1EE53345327003020D31
:100C9E001EE490E68AF090E68BF090E6A0E020E16C
:100CAE00F990E68BE0753400F53590E6B9E0B4A323
:100CBE0036E4F536F537C3E5379535E536953450D8
:100CCE003374402537F58274E73536F583E0FFE55A
:100CDE00312537F582E5303536F583EFF00537E50A
:100CEE003770D3053680CFAD357AE77B40AF31AE66
:100CFE0030121E37E5352531F531E5343530F53016
:100D0E00C3E5339535F533E5329534F532020C965D
:010D1E0022B2
:0B22FA00E54645457003D38001C32278
:02232900D322BD
:02232B00D322BB
:0800030090E6BAE0F543D322B8
:10229B0090E740E543F0E490E68AF090E68B04F09B
:0222AB00D3223C
:0813F70090E6BAE0F54AD322AA
:1022AD0090E740E54AF0E490E68AF090E68B04F082
:0222BD00D3222A
:02232D00D322B9
:02232F00D322B7
:02233100D322B5
:10119500E4FF90E6B8E020E7030212730F0F7440F6
:1011A5002401F582E434E7F5837409F00F744024D3
:1011B50002F582E434E7F583E4F00F74402403F587
:1011C50082E434E7F583E4F00F74402404F582E407
:1011D50034E7F5837404F00F74402405F582E43494
:1011E500E7F5837404F00F74402406F582E434E7D0
:1011F500F583E4F00F74402407F582E434E7F583C2
:10120500E4F00F74402408F582E434E7F58374FFB5
:10121500F00F74402409F582E434E7F58374FFF098
:101225000F7440240AF582E434E7F5837408F00F5F
:101235007440240BF582E434E7F5837420F00F74D1
:1012450040240CF582E434E7F583741FF00F7440F5
:10125500240DF582E434E7F583741FF090E740EF41
:0E126500F0E490E68AF090E6BEE090E68BF0B2
:011273002258
:100E5A0090E6B9E01203A00EA1100EA1110ECF1454
:100E6A000F40150E8F280E892E0E833C0E9B3F0EC7
:100E7A0095A20E95A300000F7A1203F2020F7C12BC
:100E8A000D1F020F7C121351020F7C120B7E020FF0
:100E9A007C121195020F7C90E6B8E030E70C7B01DA
:100EAA007AE7794012000E020F6490E6BEE090E6FF
:100EBA008BF090E6A0E020E1F97B017AE779401215
:100ECA001F64020F7CE4F52C74A9252CF582E43406
:100EDA0028F583E0FF7440252CF582E434E7F58396
:100EEA00EFF0052CE52CB404DFE4F52C74B3252CC3
:100EFA00F582E43428F583E0FF7444252CF582E476
:100F0A0034E7F583EFF0052CE52CB404DFE4F52C87
:100F1A0074AF252CF582E43428F583E0FF74482564
:100F2A002CF582E434E7F583EFF0052CE52CB404C4
:100F3A00DF121F928024E4F52C7485252CF582E4B7
:100F4A003428F583E0FF7440252CF582E434E7F574
:100F5A0083EFF0052CE52CB404DFE490E68AF090E8
:100F6A00E6BEE090E68BF090E6A0E04480F08002D6
:030F7A00C322D3BC
:010F7D002251
:1020E100C0E0C083C08290E6B5E04401F0D2015364
:0F20F10091EF90E65D7401F0D082D083D0E032A1
:10224800C0E0C083C0825391EF90E65D7404F0D083
:0622580082D083D0E032C9
:10225E00C0E0C083C0825391EF90E65D7402F0D06F
:06226E0082D083D0E032B3
:101D9300C0E0C083C08290E680E030E70E85090D85
:101DA300850A0E85110F851210800C85110D851281
:101DB3000E85090F850A105391EF90E65D7410F0BC
:071DC300D082D083D0E03292
:10223000C0E0C083C082D2035391EF90E65D740882
:08224000F0D082D083D0E0321F
:101DCA00C0E0C083C08290E680E030E70E85090D4E
:101DDA00850A0E85110F851210800C85110D85124A
:101DEA000E85090F850A105391EF90E65D7420F075
:071DFA00D082D083D0E0325B
:012339003271
:01233A003270
:01233B00326F
:01233C00326E
:01233D00326D
:01233E00326C
:01233F00326B
:01234000326A
:012341003269
:012342003268
:012343003267
:012344003266
:012345003265
:012346003264
:012347003263
:012348003262
:012349003261
:01234A003260
:01234B00325F
:01234C00325E
:01234D00325D
:01234E00325C
:01234F00325B
:01235000325A
:012351003259
:012352003258
:012353003257
:012354003256
:012355003255
:012356003254
:012357003253
:012358003252
:012359003251
:01235A003250
:01235B00324F
:01235C00324E
:10217500E4F5C8E58E54074438F58E8FCB8FCDAF87
:0C218500058FCA8FCCD2BDD2ADD2CA22C9
:101F0400AB07AA06A905A8047F007E1B7D377C4B7E
:101F1400120151AB07AA06A905A804E4FFFE7D80BF
:101F24007C4712005912022CAD07AC06AF04022103
:011F34007537
:1022BF00AD07AC06C3E49DFBE49CFFEBFD0221756B
:03232600C2CA2206
:03002B00021CA212
:101CA200C0E0C0F0C083C082C0D075D000C000C008
:101CB20001C002C003C004C005C006C0071222ED65
:101CC200C2CFD007D006D005D004D003D002D001B5
:0D1CD200D000D0D0D082D083D0F0D0E0324E
:0A23050000010202030304040505B1
:03000B00021B4293
:101B4200C0E0C0F0C0D075D000C000C004C005C065
:101B520006C0070508E508B406210559E5597002D3
:101B62000558AE58FF7C007D0A120327ED4C700821
:101B7200054CE54C7002054B750800D007D006D025
:0C1B820005D004D000D0D0D0F0D0E0326C
:1015E600E4F528F527F526F525C203C200C202C296
:1015F60001121D57750B0F750C7E75130F75149020
:1016060075090F750A9A75110F7512BA75150F754A
:1016160016DAD2E843D82090E668E04409F090E66E
:101626005CE0443DF0D2AFD208121F3590E680E070
:1016360054F7F0C203300105120959C201300329DB
:101646001222FA5024C20312201620001690E682B7
:10165600E030E704E020E1EF90E682E030E604E0E7
:0E16660020E0E4121FBE12232912211E80C7AD
:1009590090E6B9E07003020A0A147003020A8724B8
:10096900FE7003020B0A24FB7003020A04147003CD
:100979000209FE14607314607624056003020B6A91
:1009890012232B4003020B7690E6BBE024FE602283
:1009990014603324FD601114602224067048E50BAD
:1009A90090E6B3F0E50C8037E51390E6B3F0E51473
:1009B900802DE50D90E6B3F0E50E8023E50F90E676
:1009C900B3F0E510801990E6BAE0FF121FEAAA0613
:1009D900A9077B01EA494B600DEE90E6B3F0EF9071
:1009E900E6B4F0020B76020B6F1222AD020B7612FF
:1009F90013F7020B76120003020B7612229B020BED
:100A09007612232D4003020B7690E6B8E0247F602E
:100A19001514601924027063A200E43325E0FFA2D3
:100A290002E4334F8041E490E740F0803F90E6BC18
:100A3900E0547EFF7E00E0D394807C0040047D0179
:100A490080027D00EC4EFEED4F2405F58274233EB5
:100A5900F583E493FF3395E0FEEF24A1FFEE34E63E
:100A69008F82F583E0540190E740F0E4A3F090E62B
:100A79008AF090E68B7402F0020B76020B6F122358
:100A89002F4003020B7690E6B8E024FE601624029C
:100A99006003020B7690E6BAE0B40105C200020BCE
:100AA90076020B6F90E6BAE0705590E6BCE0547E92
:100AB900FF7E00E0D394807C0040047D0180027DAC
:100AC90000EC4EFEED4F2405F58274233EF583E4D8
:100AD90093FF3395E0FEEF24A1FFEE34E68F82F514
:100AE90083E054FEF090E6BCE05480131313541FC6
:100AF900FFE0540F2F90E683F0E04420F0806E80F1
:100B090065122331506790E6B8E024FE601A24028A
:100B1900705B90E6BAE0B40104D200805090E6BA66
:100B2900E0B402028047803E90E6BCE0547EFF7E3E
:100B390000E0D394807C0040047D0180027D00ECBC
:100B49004EFEED4F2405F58274233EF583E493FFB1
:100B59003395E0FEEF24A1FFEE34E68F82F5838022
:100B6900081206FD500790E6A0E04401F090E6A0C7
:040B7900E04480F0E4
:010B7D002255
:0300330002231F86
:04231F0053D8EF326E
:101FBE0090E682E030E004E020E60B90E682E0302E
:101FCE00E119E030E71590E680E04401F07F147EE1
:0C1FDE0000121BD990E680E054FEF022B7
:1020160090E682E044C0F090E681F043870100003C
:042026000000002294
:101F350030080990E680E0440AF0800790E680E0EA
:101F45004408F07FDC7E05121BD990E65D74FFF036
:0F1F550090E65FF05391EF90E680E054F7F022B2
:08230F00E4F51CD2E9D2AF2273
:101E010090E678E020E6F9C2E990E678E04480F0D7
:101E1100EF25E090E679F090E678E030E0F990E6A1
:101E210078E04440F090E678E020E6F990E678E04A
:061E310030E1D6D2E922E7
:101ED200A90790E678E020E6F9E51C702390E67801
:101EE200E04480F0E925E090E679F08D17AF03A990
:101EF200077518018A19891AE4F51B751C01D3228A
:021F0200C322F8
:101E6C00A90790E678E020E6F9E51C702590E67865
:101E7C00E04480F0E925E0440190E679F08D17AF5D
:101E8C0003A9077518018A19891AE4F51B751C0337
:041E9C00D322C32268
:03004B0002108D13
:10108D00C0E0C083C082C085C084C086758600C0A4
:10109D00D075D000C000C001C002C003C006C0079B
:1010AD0090E678E030E206751C0602117790E6783E
:1010BD00E020E10CE51C64026006751C0702117747
:1010CD00E51C24FE605F14603624FE700302116877
:1010DD0024FC700302117424086003021177AB180D
:1010ED00AA19A91AAF1B051B8F827583001202C6A0
:1010FD0090E679F0E51B65177070751C05806B9097
:10110D00E679E0AB18AA19A91AAE1B8E8275830079
:10111D00120305751C02E5176401704E90E678E028
:10112D004420F08045E51724FEB51B0790E678E0D6
:10113D004420F0E51714B51B0A90E678E04440F022
:10114D00751C0090E679E0AB18AA19A91AAE1B8E92
:10115D0082758300120305051B800F90E678E0442D
:10116D0040F0751C008003751C005391DFD007D033
:10117D0006D003D002D001D000D0D0D086D084D0FC
:08118D0085D082D083D0E0324E
:021FEA00A90745
:101FEC00AE15AF168F828E83A3E064037017AD011C
:101FFC0019ED7001228F828E83E07C002FFDEC3E68
:09200C00FEAF0580DF7E007F00BD
:0120150022A8
:10219100121E6CE51C24FA600E146006240770F30D
:0C21A100D322E4F51CD322E4F51CD32269
:1021AD00121ED2E51C24FA600E146006240770F38B
:0C21BD00D322E4F51CD322E4F51CD3224D
:101BD9008E298F2A90E600E054187012E52A240114
:101BE900FFE43529C313F529EF13F52A801590E68B
:101BF90000E05418FFBF100BE52A25E0F52AE52976
:101C090033F529E52A152AAE29700215294E6005F2
:061C190012202A80EE22D9
:10202A007400F58690FDA57C05A3E582458370F9C9
:01203A002283
:03004300021400A4
:0300530002140094
:101400000220E10002225E00022248000222300097
:10141000021D9300021DCA000223390002233A0074
:1014200002233B0002233C0002233D0002233E0036
:1014300002233F0002234000022341000223420016
:101440000223430002233A00022344000223450002
:1014500002234600022347000223480002234900DA
:1014600002234A0002233A0002233A0002233A00F0
:1014700002234B0002234C0002234D0002234E00A6
:1014800002234F0002235000022351000223520086
:101490000223530002235400022355000223560066
:1014A00002235700022358000223590002235A0046
:0814B00002235B0002235C0033
:10005600020298E86480F8E933E83360110460F03E
:10006600ED33EC337009E8FCE9FDEAFEEBFF220410
:1000760060DED3EB9FEA9EE99DE8C2E78CF0C2F70B
:1000860095F0400CE8CCF8E9CDF9EACEFAEBCFFBD7
:1000960012026385D0F05804700320D5B3E80470CB
:1000A600075002B2D50202A292D5EC0460F7E4CC66
:1000B600C0E0C398F8603B94186008400DD0E0FBA0
:1000C60002027AE4FBFAC9FC8028E830E406E4C9B7
:1000D600FBE4CAFCE830E305E4C9CACBFCE85407F4
:1000E6006010F8C3E913F9EA13FAEB13FBEC13FCFF
:1000F600D8F130F52FC3E49CFCEF9BFFEE9AFEEDA2
:1001060099FDD0E0FBEF4E4D4C701222DB0302024C
:100116009FEC2CFCEF33FFEE33FEED33FDED30E7C5
:10012600EB02027AEF2BFFEE3AFEED39FDD0E0FB53
:1001360050130BBB00030202A2ED13FDEE13FEEFFC
:0801460013FFEC13FC02027A26
:10014E000202A2EC5D046005E859047003020298F5
:10015E00120263580460F6EC4860F2EC7004FDFE87
:10016E00FF22C860DB2481C85009C3986002500684
:10017E0002029F9850CAF582E9294B4A7005AB825C
:10018E0002028E75F0007C1A7880C3EF9BEE9AED1A
:10019E0099400DC3EF9BFFEE9AFEED99FDE842F0FC
:1001AE00DC23ACF0D0E0FFD0E0FED0E0FDAB82204F
:1001BE00E7101BEB60BAEC2CFCEF33FFEE33FEEDD9
:1001CE0033FD02027AE803F830E705C0F075F0005F
:1001DE00EF2FFFEE33FEED33FD40B830E7C280AABD
:1001EE0075F020800E75F010800575F0087D007E8C
:1001FE00007F003392D530D503120392EC334010BA
:10020E00EF33FFEE33FEED33FDEC33FCD5F0ED2294
:0E021E00E5F0247EA2D513CC92E7CDCEFF22D0
:10022C00EDD2E7CD33EC3392D524814006E4FFFECA
:10023C00FDFC22FCE4CFCECDCC24E0501174FF8029
:10024C00EDC3CC13CCCD13CDCE13CECF13CF0470C6
:07025C00F030D5DE02039231
:10026300E9D2E7C933E833F892D5EDD2E7CD33ECE1
:0702730033FC5002B2D5225A
:10027A00EC30E7100FBF000C0EBE00080DBD0004E5
:10028A000BEB6014A2D5EB13FCED92E7FD2274FF91
:10029A00FCFDFEFF22E480F8A2D574FF13FC7D80EA
:0302AA00E480EFFE
:0300000002167471
:0C167400787FE4F6D8FD7581650216BB96
:1002AD00BB010689828A83E0225002E722BBFE024F
:0902BD00E32289828A83E4932282
:1002C600BB010CE58229F582E5833AF583E02250ED
:1002D60006E92582F8E622BBFE06E92582F8E22237
:0D02E600E58229F582E5833AF583E4932251
:1002F300BB010689828A83F0225002F722BBFE01EA
:02030300F322E3
:10030500F8BB010DE58229F582E5833AF583E8F02E
:10031500225006E92582C8F622BBFE05E92582C8DA
:02032500F222C2
:10032700BC000BBE0029EF8DF084FFADF022E4CCBA
:10033700F875F008EF2FFFEE33FEEC33FCEE9DEC83
:10034700984005FCEE9DFE0FD5F0E9E4CEFD22EDC9
:10035700F8F5F0EE8420D21CFEADF075F008EF2F13
:10036700FFED33FD4007985006D5F0F222C398FD04
:050377000FD5F0EA22A1
:10037C00C5F0F8A3E028F0C5F0F8E582158270020C
:06038C001583E038F022A9
:0E039200C3E49FFFE49EFEE49DFDE49CFC227C
:1003A000D083D082F8E4937012740193700DA3A3EC
:1003B00093F8740193F5828883E473740293686000
:0603C000EFA3A3A380DF00
:101AA0008B308A318932E4F538F539E5371537AEB0
:101AB00036700215364E6033AB33AA34A9351202A4
:101AC000ADFFAB30AA31A9320539E539AC38700227
:101AD000053814F5828C83EF120305EF60CD740195
:101AE0002535F535E43534F53480C0AB30AA31A95D
:021AF0003222A0
:10227400E4FFFE1202AD600C0FEF70010E09E9706D
:05228400F20A80EF22C8
:1003C600EF4E6012EF60010EEDBB010B89828A834E
:1003D600F0A3DFFCDEFA2289F05007F709DFFCA95B
:0C03E600F022BBFEFCF309DFFCA9F022B2
:101680000215E6E493A3F8E493A34003F68001F285
:1016900008DFF48029E493A3F85407240CC8C3336B
:1016A000C4540F4420C8834004F456800146F6DF3A
:1016B000E4800B010204081020408090213CE47E6D
:1016C000019360BCA3FF543F30E509541FFEE4932F
:1016D000A360010ECF54C025E060A840B8E493A3F6
:1016E000FAE493A3F8E493A3C8C582C8CAC583CA21
:1016F000F0A3C8C582C8CAC583CADFE9DEE780BED9
:012158000086
:00000001FF
